:10000000020688C0E0C006C0072005127E4B7F466E
:10001000B296DFFEDEF8C296E54F6002D296D007B8
:10002000D006D0E022853C35853D36AE4EBE000A76
:100030002536F536E5F03535F535C3E5459536E534
:100040004495354008E5369543E53595422275F0EF
:10005000FF74FF800575F0007401755C20120003C9
:10006000755800755900AF4EBF0002802CC0E0C02B
:10007000F075F006A4254CB4EA03E48005B4FA0256
:1000800074E4F54C1204C7200603120025D0F0D00A
:10009000E040DA1204B302049DC0F0854DF0A4D014
:1000A000F0C0E0200603120025D0E0401EC0E0C0F2
:1000B000F0253FF53FE5F0353EF53ED0F0D0E025A8
:1000C0003DF53DE5F0353CF53C801FE5F0B4000E14
:1000D00085423E85423C85433F85433D800C8544B7
:1000E0003E85443C85453F85453D22E53375F01905
:1000F000A4F533C0F0E53275F019A485F034D0F0E2
:1001000025F0C0D0F532E53175F019A48534F0D072
:10011000D035F0F531228550358551367B02C3E567
:100120003633F536E53533F535DBF31203D430E4F9
:1001300008853C37853D388006853E37853F3875D4
:1001400031008537328538331200EB1203D430E4A6
:100150000DC3E538954BF538E537954AF537C3E5D6
:100160003833F538E53733F537E53633F536E535E9
:1001700033F5357835E612024E08B839F80000D26A
:020180009500E8
:1001820000C295120504855C2875B074209208752A
:10019200215475227880067521527522783007061F
:1001A20075214675226EE53EB53C07E53FB53D0239
:1001B2008003752652E54045416003752774E54E7C
:1001C2006015E54C75F006840475F00A844430F538
:1001D20024E5F04430F5257829760008B831FAC3D1
:1001E2007C1878337D08E633F618DDFADC2F782D9B
:1001F20012023F8F2912023F8E2A8F2B12023F8E4C
:100202002C8F2D12023F8E2E8F30752F2E748078F8
:1002120021120380E61203A108B831F822783012C5
:100222000230782F120230782E12023080B474031A
:100232002630E301F674302630E701F622E6C45494
:100242000F4430FEE6540F4430FF08227C08C333CB
:1002520092B000D2B100C2B1DCF5227C10900E182F
:10026200748012051A900E28120516E4F55A900FA2
:1002720010FA7C067B011202BB900F16FA7C067BF9
:10028200261202BBE4755A02900F32FA7C067B01F9
:100292001202BB900F38FA7C067B261202BB755AFB
:1002A20000900F1C7AEA7C167B011202BB755A027F
:1002B200900F3E7AEA7C167B01E4C004C0E093F51D
:1002C20057EA1202D2D0E0040ADCF1D004DBEA22BF
:1002D200C0E0C0E01202F4E55A44A012030AD0E0E2
:1002E20012030AE55712030A12036ED0E07D1A02C6
:0602F20003BC75B0FF0023
:1002F800C2B7120333D2B7120333C2B0120333C2E8
:10030800B7227D0875B07E331203334007C2B0129E
:1003180003338005D2B0120333D2B7120333DDE4BE
:10032800120333C2B712033375B0FF7F040203B957
:10033800F5F01202F4E55A44A012030AE5F012039C
:100348000A1202F4E55A44A112030A7D08C2B71240
:100358000333D2B712033320B003C38001D3C2B72B
:1003680012033333DDE7C2B7120333C2B0120333CB
:10037800D2B7120333D2B022C4C0E054EF44E0F540
:10038800B00000C2B51203BCD0E0C454EF44E0F59D
:10039800B00000C2B5801D7420C4C0E044F0F5B0C0
:1003A8000000C2B5D0E0C444F0F5B00000C2B57F8B
:1003B80014DFFE227E371203B7DEFB227403F5B08A
:1003C800C0E0D2B5D0E0C2B57E0080EAE47DF72374
:1003D8008DB000309201041DBDEFF47D28DDFE22B2
:1003E800E55AC0E0755A0074FE120338F55074FFE0
:1003F800120338F551D0E0F55A784F74FDC0E01279
:100408000338F618D0E014B4EFF3AB4EBB000F7B03
:1004180006C0E0120338F618D0E014DBF422E54CED
:10042800240580EB1203D464FF54F770F78085E548
:100438004E701D74EA853C571202D204853D57124E
:1004480002D204853E571202D204853F570202D2D7
:1004580074FA854C570202D2E54E702C74EAC0E05B
:0304680012033844
:10046B00F53CD0E004C0E0120338F53DD0E004C009
:10047B00E0120338F53ED0E004120338F53F754027
:10048B00007541002274FA120338F54C1204C7129E
:10049B0004B3E54C04040404C0E0120338F540D067
:1004AB00E004120338F54122E54C0404C0E01203CA
:1004BB0038F53ED0E004120338F53F22E54CC0E09E
:1004CB00120338F53CD0E004120338F53D22853C8D
:1004DB0057E54C1202D204853D571202D204853ED9
:1004EB00571202D204853F571202D204854057128D
:1004FB0002D2048541570202D27821762008B83106
:10050B00FA227C1074C012038080157C1074C01208
:10051B00038074009360091203A1DC0122A380F213
:10052B0074201203A1DCF9221200551201167B6014
:10053B001203BC1203D44408B4FF051203BC801A87
:10054B001203B7DBEB1200551201167B0A1203BC28
:10055B00DBFB1203D4B4FFED80E62212004E120136
:10056B00167B601203BC1203D4B4FF051203BC80CC
:10057B001A1203B7DBED12004E1201167B0A12039F
:10058B00BCDBFB1203D4B4FFED80E6227853900D55
:10059B003AE55293F6A308B857F722758921C28E14
:1005AB00758DFF758BBCD294D28E30B6FDC28EC2C8
:1005BB009474C0120380E55A0324411203A1E58B06
:1005CB007C0C755B00C394C0403603541F6031FB39
:1005DB00941E40027B1DEBF55B13C0D0540F6013D0
:1005EB00FB74C112038074081203A1DC04D0D08009
:1005FB000CDBF3D0D0500674071203A11CEC600780
:10060B0074201203A1DCF9E55B6026C3940E502B1A
:10061B0074CD120380E55B13C0D054072432120350
:10062B00A1D0D05004742B800274201203A10203BA
:10063B009F74CD12038012039F80EEC0E074CD1225
:10064B00038074391203A174CE120380900DD6D09F
:10065B00E023C0E0931203A1D0E004930203A1793D
:10066B00051203BCD9FB2275F010900EB874401222
:10067B0003807400931203A1A3D5F0F622C2AF75C9
:10068B00815D7590FF75B0FF1203C41203C4120392
:10069B00C474021203C67428120380740C120380F4
:1006AB0074281203807401120380755A0274FF12AE
:1006BB000338F5F054F0B4A0061203D420E703126C
:1006CB00025D75815DD297C207C206C205755A02DB
:1006DB0074FF1203385402F55A1203E8755C207547
:1006EB00F048900EC812067812050DD29775580077
:1006FB00755900120116E558B4FF1D1205A6120319
:10070B00D430E01630E11630E21630E41630E51541
:10071B0030E61530E71580DE80140207B10207E6DC
:10072B000208A3802002081B020886020905E5596E
:10073B002401F559E5583400F558B401067558FFF6
:10074B0012043780B6120672120116E54F600AD2F8
:10075B0096900DF61205168008C296900E0712059C
:10076B0016758911C29775B074E5406014B293C2C7
:10077B008E85408D85418BD28E209225108FEE80F9
:10078B00FB75B077209214B293C28E758DFF758B6B
:01079B001548
:10079C00D28E209205108FEE80FB75B0743092E0F3
:1007AC00D2970206EA1200551201167B901203BC76
:1007BC001203D44408B4FF061203BC0206EA120367
:1007CC00B7DBEA1200551201167B301203BCDBFBBF
:1007DC001203D44408B4FFEB80E412004E1201164D
:1007EC007B901203BC1203D44408B4FF061203BC62
:1007FC000206EA1203B7DBEA12004E1201167B3036
:10080C001203BCDBFB1203D44408B4FFEB80E412EC
:10081C0000031204377F327E001EDE051FDFF880D6
:10082C00251203D464FF54F770EF12042C1203BC8E
:10083C00755C20E54EB2E0F54EF55774FC1202D211
:10084C001204600206EAE54E60E0E55CB4720F75D6
:10085C005C2012046012011612042C0206EA755C6C
:10086C0072AE3EAF3C8F3E8E3CAE3FAF3D8F3F8E67
:10087C003D12011612042C0206EA120437755A02B4
:10088C001203BC74FF120338B2E1F55774FF120265
:10089C00D212042C0206CD120003D20512042C90A5
:1008AC000E391205167AFF1200551203D4FB54F7B9
:1008BC00B4F73BC3E549953DE548953C40E9E53D3A
:1008CC009547E53C954640DF120116791E1203BC94
:1008DC001203BC1203D4FB54F7B4F712EB30E3044D
:1008EC00D9EB80B31205A61203BCDADF80B1C205C6
:1008FC0012000312042C0206EA12050D120437D260
:10090C0007E4F54E12011612042C1203D430E01D2C
:10091C0030E11A30E21930E41830E50B30E60B30D8
:10092C00E70280E6020D31020A4D020C918025800F
:10093C006D120672E54F6014754F00900E0712058C
:10094C0016854F5774FD1202D2020D31754FFF9070
:04095C000DF680EA2A
:1009600012042CE54D75F019A475310085F032F5AF
:1009700033120185900E451205161203D430E0089B
:1009800030E10F30E71680F2120003E54D04F54D1B
:1009900080CE120003E54D14F54D80C474FB854DE7
:1009A000571202D2120003020D3185463C85463EA5
:1009B00085473D85473FC20512000312042C1201F2
:1009C00016900E4A1205161203D430E00830E110DA
:1009D00030E71880F2120533853C46853D4780DBC1
:1009E000120566853C46853D4780D085483C854854
:1009F0003E85493D85493F12000312042C12011621
:100A0000900E571205161203D430E00830E1103072
:100A1000E71880F2120533853C48853D4980DB129A
:100A20000566853C48853D4980D074F4854657125B
:100A300002D2048547571202D2048548571202D2C7
:100A4000048549571202D2120003020D311200032D
:100A5000D206E4F54C04F54E900E841205161204ED
:100A6000C71204B312049D12011612042C1203D4EF
:100A700030E00830E11430E72180EF120003E54C4C
:100A80002406B4EA01E4F54C80CE120003E54C9450
:100A900006B4FA0274E4F54C80BE120003900E8D89
:100AA00012051612011612042C1203D430E00B307A
:100AB000E14C30E70280EF020B47E53D2401F53DB4
:100AC000F53FE53C3400F53CF53E120116120003FB
:100AD0007C1E1203D420E0C512066ADCF5E53D2435
:100AE00001F53DF53FE53C3400F53CF53E120116BD
:100AF0001200031203D420E0A412066A80DFC3E5CB
:100B00003D9401F53DF53FE53C9400F53CF53E1282
:100B100001161200037C1E1203D420E12712066A7C
:070B2000DCF5C3E53D940183
:100B2700F53DF53FE53C9400F53CF53E1201161204
:100B370000031203D420E10512066A80DE020A9D33
:100B4700900E9A120516E53C853E3CF53EE53D853F
:100B57003F3DF53F12011612000312042C1203D475
:100B670030E00A30E14330E70280EF807DE53D2445
:100B770001F53DE53C3400F53C1201161200037CFB
:100B87001E1203D420E0D312066ADCF5E53D2401EA
:100B9700F53DE53C3400F53C120116120003120343
:100BA700D420E0B612066A80E3C3E53D9401F53D23
:100BB700E53C9400F53C1201161200037C1E12035B
:100BC700D420E12312066ADCF5C3E53D9401F53D27
:100BD700E53C9400F53C1201161200031203D420E1
:100BE700E10512066A80E2020B61E53C853E3CF5B1
:100BF7003EE53D853F3DF53F900EA7120516755220
:100C070000900D3A7853E55293F6A308B857F7E5E5
:100C170040C395557007E541C39556600FE55224CB
:100C270004F552B59CDB7552001200031205977547
:100C3700310085533285543385554085564112011D
:100C47008512042C1203D430E00B30E11730E53164
:100C570030E72280EC120003E5522404B49C01E43F
:100C6700F55280C8120003C3E5529404B4FC027421
:100C770098F55280B71204D912000312042C020A05
:100C8700581204D9120003020D31D20685423C8561
:100C9700423E85433D85433F12000312042C120157
:100CA70016900E651205161203D430E00830E110D5
:100CB70030E71880F2120533853C42853D4380DBDF
:100CC700120566853C42853D4380D085443C85447A
:100CD7003E85453D85453F12000312042C1201163F
:100CE700900E741205161203D430E00830E110306C
:100CF700E71880F2120533853C44853D4580DB12B9
:100D07000566853C44853D4580D074F08542571281
:100D170002D2048543571202D2048544571202D2E5
:100D2700048545571202D212000312042C1203BC89
:100D37000206CD00000000029EE72702CFE8D90295
:100D4700E8E9A00302EA62031DEB1D0339EBD303B5
:100D570056EC830375ED320393EDD003B4EE7203C3
:100D6700CEEEEA03E8EF5C040BEFEC0430F07B0413
:100D770055F100047CF18204A4F1FF04CEF27A0459
:100D8700F9F2EF0526F3620555F3D10585F43B0526
:100D9700B6F4A005EAF505061FF5640656F5C00684
:100DA7008FF61A06CAF6700707F6C30746F7130742
:100DB70088F76207F3F7D6083BF81E0885F863083B
:100DC700D1F8A40920F8E40972F92209C7F95E05E8
:100DD70005050305060105010301060205020302D5
:100DE700060305030303060405040304062B2B016E
:100DF700010101010101010101202020486967006B
:100E0700010101010120202020202020204C6F77A4
:100E17000020496E697469616C697A6174696F6EE3
:100E2700004275696C64202D2032312E30382E3007
:100E370035005363616E6E696E672E2E2E005374F4
:100E47006570005363616E6E696E67204C6F770043
:100E57005363616E6E696E67204869676800426117
:100E67006E64204C6F77206C696D69740042616E07
:100E7700642048696768206C696D6974004368611C
:100E87006E6E656C73005278204672657175656E7B
:100E97006379005478204672657175656E637900D1
:100EA700537562546F6E65202043682D45786974C9
:100EB7000000000000000000000000001F1F1F1FAF
:100EC7000000000000000000000000010301010114
:100ED700000000060902040F0000000F0102010FC5
:100EE70000000003050F01010000000609090906BB
:100EF70000000006080E0906000000001818181860
:100F0700000000001B1B1B1B00E308E3080000E4B4
:100F17002AE42A0000E308E3080000E100E420E1F6
:100F2700C8E3D010B6000A00001000E308E3080089
:100F370000E42AE42A0000E308E3080000E100E4F3
:0D0F470020E1C8E3D010B6000A0000FFA0B2
:00000001FF
